:100000000C9438000C9466000C94FC000C94530083
:100010000C9453000C9453000C9453000C94530014
:100020000C9453000C9453000C9453000C94530004
:100030000C9453000C9453000C9453000C945500F2
:100040000C9453000C9453000C9453000C945300E4
:100050000C9453000C9453000C9453000C945300D4
:100060000C9453000C9453000C9453000C945300C4
:1000700011241FBECFEFD0E1DEBFCDBF12E0A0E064
:10008000B1E0E6E9F0E102C005900D92AE38B107AB
:10009000D9F71FE0AEE8B2E001C01D92AD3FB10755
:1000A000E1F70C9470040C9400001F920F920FB6AD
:1000B0000F9211248F9380918E028F5F80938E0216
:1000C0008F910F900FBE0F901F9018951F920F9257
:1000D0000FB60F9211246F937F938F939F93EF939B
:1000E000FF93E0918F02FF2780918400909185001B
:1000F000EE0FFF1FE356FD4F91838083E0918F0247
:10010000FF2780918E02E353FD4F8083E0918F02A1
:10011000FF2780913701F695FE2FEE27F795E7959B
:10012000EB51FD4F8587E0918F02FF2780913801C9
:10013000F695FE2FEE27F795E795EB51FD4F868755
:10014000E0918F02FF2780913901F695FE2FEE276F
:10015000F795E795EB51FD4F8787E0918F02FF27D9
:1001600080913A01F695FE2FEE27F795E795EB5132
:10017000FD4F808BE0918F02FF2780913B01F69528
:10018000FE2FEE27F795E795EB51FD4F818BE09120
:100190008F02FF2780913C01F695FE2FEE27F79501
:1001A000E795EB51FD4F828BE0918F02FF27EB51DA
:1001B000F14F85E5808380918F028F5F80938F025E
:1001C00080918F0268E10E943F0890938F02809196
:1001D00091028F5F8093910280919102843009F4A3
:1001E000E898FF91EF919F918F917F916F910F9080
:1001F0000FBE0F901F9018951F920F920FB60F927F
:1002000011242F933F934F935F936F937F938F931B
:100210009F93AF93BF93EF93FF9387E788B988B914
:100220008FEF88B986B18171E9F3E0918F02FF27E2
:100230008091840090918500EE0FFF1FE356FD4FE3
:1002400091838083E0918F02FF2780918E02E35398
:10025000FD4F808386B18171E9F789E988B988B952
:1002600088B988B940B193B18FEF88B920E030E008
:1002700077E76FEF59E9EDEFFEE078B978B968B943
:1002800086B18171E9F3408391832E5F3F4F3296AF
:1002900086B18171E9F758B958B958B958B940B120
:1002A00093B168B92E3F310541F74093FB0F90930E
:1002B000FC0F80919C02833009F486C080919C02DF
:1002C0008823A9F59091FD0E97FDB3C08091FE0E95
:1002D00087FDCEC0981708F08FC040E050E0ADEF2A
:1002E000BEE0E0918F02FF27CA01969587952C9179
:1002F0001296F695FE2FEE27F795E795EB51FD4FF9
:10030000E80FF91F20834E5F5F4F81E040305807B0
:1003100041F7E0918F02FF27F695FE2FEE27F79524
:10032000E795EC59FC4F80818E7F80832EC08091B1
:100330009C02813009F47FC041E050E0AEEFBEE0A6
:10034000E0918F02FF27CA01969587952C9112960E
:10035000F695FE2FEE27F795E795EB51FD4FE80F49
:10036000F91F20834E5F5F4F81E04130580741F70E
:10037000E0918F02FF27F695FE2FEE27F795E79580
:10038000EC59FC4F808181608083E0918F02FF27D0
:10039000EB51F14F8AEA808380918F028F5F8093C7
:1003A0008F0280918F0268E10E943F0890938F0234
:1003B000809192028F5F80939202809192028431A9
:1003C00009F058C0E99856C020E030E0ADEFBEE03B
:1003D000E0918F02FF278D91F695FE2FEE27F7957E
:1003E000E795EB51FD4FE20FF31F80832F5F3F4FE7
:1003F0002038310569F7C9CF41E050E0AEEFBEE0EB
:10040000E0918F02FF27CA01969587952C9112964D
:10041000F695FE2FEE27F795E795EB51FD4FE80F88
:10042000F91F20834E5F5F4F81E04130580741F74D
:100430009FCF90954BCF40E050E0ADEFBEE0E09114
:100440008F02FF27CA01969587952C911296F695F3
:10045000FE2FEE27F795E795EB51FD4FE80FF91FBB
:1004600020834E5F5F4F81E04030580741F751CF06
:10047000809530CF82E08CBBFF91EF91BF91AF911F
:100480009F918F917F916F915F914F913F912F91AC
:100490000F900FBE0F901F9018958F708A3018F034
:1004A000895C99270895805D99270895982F8091F8
:1004B000C00085FFFCCF9093C6000895DC01EC914D
:1004C000EE2371F090E08091C00085FFFCCFE093B7
:1004D000C6009F5FFD01E90FF11DE081EE2399F752
:1004E00008951F93182F8091C00085FFFCCF812FA6
:1004F00082958F700E944D028093C6008091C0004B
:1005000085FFFCCF812F0E944D028093C6001F9172
:100510000895CF93DF93EC018091C00085FFFCCF5D
:10052000CE01892F992782958F700E944D0280936A
:10053000C6008091C00085FFFCCF8D2F99270E94B7
:100540004D028093C6008091C00085FFFCCFCE0194
:10055000929582958F7089279F7089270E944D02FE
:100560008093C6008091C00085FFFCCF8C2F0E9435
:100570004D028093C600DF91CF91089560E070E056
:1005800020E030E040E050E089B18F7E8BB92F5FF2
:100590003F4F4F4F5F4F203888E3380781E04807CF
:1005A00080E0580789F720E030E040E050E089B172
:1005B00080618BB92F5F3F4F4F4F5F4F203888E3EB
:1005C000380781E0480780E0580789F720E030E0ED
:1005D00040E050E089B18F7D8BB92F5F3F4F4F4F87
:1005E0005F4F203888E3380781E0480780E05807EC
:1005F00089F720E030E040E050E089B180628BB9BB
:100600002F5F3F4F4F4F5F4F203888E3380781E01F
:10061000480780E0580789F720E030E040E050E0EC
:1006200089B18F7B8BB92F5F3F4F4F4F5F4F203882
:1006300088E3380781E0480780E0580789F720E021
:1006400030E040E050E089B180648BB92F5F3F4FCC
:100650004F4F5F4F203888E3380781E0480780E03C
:10066000580789F76F5F7F4F6430710509F088CFB5
:10067000089560E070E020E030E040E050E089B1B3
:100680008F788BB92F5F3F4F4F4F5F4F203888E3F4
:10069000380781E0480780E0580789F720E030E01C
:1006A00040E050E089B180678BB92F5F3F4F4F4FDB
:1006B0005F4F203888E3380781E0480780E058071B
:1006C00089F76F5F7F4F68307105A9F60895982FFD
:1006D00080919402873028F5292F33278091940246
:1006E000E0918102F0918202E80FF11D808199274B
:1006F00087FD90952817390709F446C041E080919D
:100700009402E0918B02F0918C02E80FF11D808140
:10071000992787FD90952817390709F44BC0442382
:1007200041F5809194028F5F8093940280919402AE
:10073000873080F01092940280919802873058F4AC
:1007400080919902873038F5109299028091990230
:100750008093980208951092990280919902809353
:100760009802809193028F5F809393021092970278
:10077000089510929402809194028093990280913E
:100780009902809398020895809198028F5F8093D8
:10079000980240E0B4CF1092990280919902809320
:1007A0009802809193028F5F8093930281E08093FF
:1007B00097020895809199028F5F80939902B1CF3B
:1007C000982F8C32A1F080919402841778F4809154
:1007D0009402262F280F312D311DF901E65DFE4FC1
:1007E0009083809194028F5F80939402089580910A
:1007F00093028F5F80939302109294020895982F32
:100800008C32F1F0809194028417C8F4903309F48B
:1008100052C080919402462F480F512D511DFA016C
:10082000E65DFE4F908381E080939B029E3209F447
:1008300054C0809194028F5F80939402089508952C
:10084000809193028F5F809393028091940284172A
:1008500058F580919A02882381F480919402262F82
:10086000280F312D311DF901E65DFE4F8EE28083A8
:10087000809194028F5F80939402809194028417F8
:1008800098F4772790E380919402FB01E80FF11D23
:10089000E65DFE4F9083809194028F5F8093940277
:1008A00080919402841778F31092940210929A0225
:1008B00010929B02089520919B02213009F0B9CF3C
:1008C00080919402462F480F512D511DFA01E65D8B
:1008D000FE4F908320939B02ACCF80939A02A9CFC6
:1008E000CFEFD0E1DEBFCDBF88E1E5EEFEE0819342
:1008F0002EE0ED3FF207D9F711B89FEF92B914B887
:1009000095B98EEE87B998B980E78AB98FE88BB927
:1009100082E08093810081E080936F0015BE8BE0C0
:100920008093690083E08DBB789480939C0289B1A9
:100930008078803809F4A1C310E080919C02833054
:1009400019F08DE480936E010E94BE02103409F408
:1009500091C3103809F48BC3112309F085C390E0CB
:100960008FE19093C5008093C40088E18093C1001B
:1009700086E08093C200E0910E01F0910F0180812A
:100980008093240180912401809367018181809369
:100990002501809125018093680182818093260141
:1009A000809126018093690180E191E00E945E02BE
:1009B000FF248091C00087FD25C080919202209184
:1009C0009102820F912D911D1816190694F7E0914E
:1009D0009002FF27EB51F14F8081853599F1E0912D
:1009E0009002FF27EB51F14F80818A3A09F45EC0F3
:1009F00080E091E00E945E020E9439038091C00075
:100A000087FFDBCF9091C60080919302882309F481
:100A10007EC180919702882309F0FFC080919302E4
:100A2000853009F4B8C2863008F091C2823009F4EA
:100A3000F4C2833008F0E6C2813009F40FC310928B
:100A40009302BBCF8091950290919602892B09F475
:100A5000F9C08091950290919602892B09F461C0AA
:100A600080919502909196020E9708F05AC080915D
:100A7000C00085FF9ECFE0919502F0919602E75D60
:100A8000FE4F80818093C600E0919502F09196021E
:100A9000E75DFE4F8081F826809195029091960245
:100AA0000196909396028093950283CF8091950250
:100AB00090919602892B09F42EC180919502909114
:100AC0009602019709F4FFC18091950290919602D8
:100AD000029708F485C18091950290919602CD9776
:100AE00008F07EC18091C00085FF63CFE091950240
:100AF000F0919602E659FE4F80818093C600E09106
:100B00009502F0919602E659FE4F8081F826809179
:100B10009502909196020196909396028093950289
:100B200048CF80919502909196020E9770F1809136
:100B3000950290919602449740F58091C00085FF00
:100B400038CF809190029927E0919502F09196021A
:100B50009695982F882797958795E80FF91FEC5160
:100B6000FD4F80818093C600809190029927E0918B
:100B70009502F09196029695982F882797958795DC
:100B8000E80FF91FEC51FD4F85CF809195029091B0
:100B90009602449740F0809195029091960282349B
:100BA000910508F464CF8091950290919602823469
:100BB000910509F4B7C18091950290919602833412
:100BC000910509F4EEC180919502909196028434CA
:100BD000910509F4ECC180919502909196028534BB
:100BE000910509F4F5C1109296021092950289B10F
:100BF00080648BB9809190028F5F80939002809186
:100C0000900268E10E943F089093900280919102C7
:100C1000815080939102E89ACCCE809193028530E6
:100C200059F0863008F0A5C1823031F0833008F0E9
:100C3000DDC1813009F003CF40E060E0892F0E94E0
:100C4000E003BBCE89B18F7B8BB9E0919002FF2787
:100C5000E353FD4F808182958F700E944D028093F7
:100C60002E01E0919002FF27E353FD4F80810E9407
:100C70004D0280932F01E0919002FF27EE0FFF1F9E
:100C8000E356FD4F80819181892F992782958F703E
:100C90000E944D0280933001E0919002FF27EE0FF9
:100CA000FF1FE356FD4F80819181892F99270E9474
:100CB0004D0280933101E0919002FF27EE0FFF1F5C
:100CC000E356FD4F80819181929582958F7089279F
:100CD0009F7089270E944D0280933201E09190021B
:100CE000FF27EE0FFF1FE356FD4F808191810E9489
:100CF0004D02809333018091950290919602019666
:100D000090939602809395024EE0F42E52CE892F56
:100D10000E94670352CE89B18F7E8BB9E091900219
:100D2000FF27E353FD4F808182958F700E944D0213
:100D300080937001E0919002FF27E353FD4F808183
:100D40000E944D0280937101E0919002FF27EE0F07
:100D5000FF1FE356FD4F80819181892F992782954E
:100D60008F700E944D0280937201E0919002FF27E4
:100D7000EE0FFF1FE356FD4F80819181892F992748
:100D80000E944D0280937301E0919002FF27EE0FC5
:100D9000FF1FE356FD4F80819181929582958F7060
:100DA00089279F7089270E944D0280937401E091EA
:100DB0009002FF27EE0FFF1FE356FD4F80819181C8
:100DC0000E944D0280937501809195029091960248
:100DD000019690939602809395025EE0F52EE9CD00
:100DE0008091950290919602CD9740F18091950265
:100DF00090919602CF9710F58091C00085FFD9CDD4
:100E0000E0919502F0919602E659FE4F8081809321
:100E1000C600E0919502F0919602E659FE4F80815E
:100E2000F82689B180618BB98091950290919602E4
:100E300001969093960280939502BBCD8091950286
:100E400090919602CF9740F08091950290919602F2
:100E50008E50914008F446CE809195029091960272
:100E60008E50914009F45EC0809195029091960257
:100E70008F50914009F495C080919502909196020F
:100E80008051914009F493C080919502909196020F
:100E90008151914009F49CC01092960210929502E3
:100EA000809190028F5F809390028091900268E120
:100EB0000E943F089093900280919202815080930B
:100EC0009202E99A76CDC0E0D0E007E711E0E09128
:100ED0009002FF27F695FE2FEE27F795E795EB5149
:100EE000FD4FEC0FFD1F808182958F700E944D0297
:100EF000F8018083E0919002FF27F695FE2FEE2700
:100F0000F795E795EB51FD4FEC0FFD1F8081219682
:100F10000E944D02F80181830E5F1F4FC038D1053A
:100F2000B1F6BACD8091C00085FF43CD8F2D82955B
:100F30008F700E944D028093C6008091950290911F
:100F400096020196909396028093950232CD873057
:100F500009F472CE873008F443C0883009F46CCEAF
:100F6000893009F06CCD46E064E1892F0E94E003EE
:100F700024CD873009F462C0873008F45DCE883014
:100F800009F45ACE893009F05ACD45E064E3892F3F
:100F90000E94FF0312CD4AE067E2892F0E94E0031E
:100FA0000CCD8091C00085FF04CD8F2DC2CF8091E4
:100FB000C00085FFFECC8DE08093C6008091950235
:100FC0009091960201969093960280939502F1CCAF
:100FD0008091C00085FFEDCC8AE08093C6005CCD97
:100FE00041E062E3892F0E94E003E7CC833009F4FB
:100FF00023CE843009F023CD40E060E0892F0E94A9
:10100000E003DBCC833021F1843009F018CD41E0DE
:1010100065E2892F0E94E003D0CC41E06BE0892F8C
:101020000E94E00380913501813471F080913C0190
:1010300080FD0AC089B180628BB9BFCC42E06AE30F
:10104000892F0E94E003B9CC89B18F7D8BB9B5CCD3
:1010500049E06BE1892F0E94E003AFCC46E06DE0F0
:10106000892F0E94E003A9CC91E083E07ACC90E044
:1010700080E477CC90E081E874CC10EE5ECC991BD4
:1010800079E004C0991F961708F0961B881F7A957F
:06109000C9F780950895E8
:101096000D0A4552524F520D0A00323943000A01D9
:1010A6000D0A4669726D77617265205665727369BD
:1010B6006F6E3A202D2D2D0D0A002442532C303010
:1010C600303030302C2D2C3030303030302C303029
:1010D600303030302C303030302E303030302C2D17
:1010E6002C30303030302E303030302C2D2C30300B
:1010F6003030302C30302C2D2D2D2A002442442C1B
:101106003030303030302C303030303030303030DD
:1011160030303030303030303030303030303030C9
:1011260030303030303030303030303030303030B9
:1011360030303030303030303030303030303030A9
:101146003030303030303030303030303030303099
:101156003030303030303030303030303030303089
:101166003030303030303030303030303030303079
:101176003030303030303030303030303030303069
:101186003030303030303030303030303030303059
:101196003030303030303030303030303030303049
:1011A6003030303030303030303030303030303039
:1011B6003030303030303030303030303030303029
:1011C6003030303030303030303030303030303019
:1011D6003030303030303030303030303030303009
:1011E60030303030303030303030303030303030F9
:1011F60030303030303030303030303030303030E9
:10120600303030303030302A00244750524D432C95
:0E1216000079022447504747412C0083020014
:00000001FF
